:03F0000002F00813
:03F0610002F003B7
:05F0030012F06480FE24
:03F0640053BEFB9D
:08F06700E5BE30E6FB53C6B81C
:0EF06F00E5C620E6FB43BE0490DF07740AF0FE
:0EF07D0090DF08E4F090DF0C7486F090DF0D59
:0EF08B007483F090DF0E7430F090DF0F74226B
:0DF09900F090DF1074F8F090DF06E4F090C6
:0EF0A600DF11F090DF1A7456F090DF1B74102B
:0EF0B400F090DF147414F090DF157416F090D5
:0EF0C200DF16746CF090DF177403F090DF1807
:0EF0D0007440F090DF197491F090DF1C74E929
:0DF0DE00F090DF1D742AF090DF1EE4F0902A
:0EF0EB00DF1F741FF090DF237488F090DF2485
:0EF0F9007431F090DF257409F090DF2E745012
:0EF10700F090DF037404F090DF047422F090A7
:0EF11500DF05E4F090DF0274FFF090DF00747D
:0BF12300AAF090DF0174AAF075E10370
:0BF12E0090DF3BE0FA53021FBA13F51C
:02F1390080FE56
:06F03700E478FFF6D8FDAD
:08F015007900E94400601B7A58
:05F01D000090F13F78B6
:03F02200007593E3
:0AF0250000E493F2A308B80002050E
:08F02F0093D9F4DAF27593FFA6
:08F03D007800E84400600A7944
:03F04500007593C0
:06F0480000E4F309D8FC0E
:08F04E007800E84400600C7931
:0BF0560000900000E4F0A3D8FCD9FA01
:03F0080075810708
:0AF00B0012F13BE582600302F003FE
:04F13B0075820022B7
:00000001FF
